:03000000020640B5
:0C064000787FE4F6D8FD75815C02068727
:1008BD00015900014400015A00014500025B00008E
:1008AA00EF1FAA0670011E4A60087D051DED60F063
:0208BA0080FAC2
:0108BC002219
:03000B00020017D9
:0100170032B6
:03001B00020018C8
:0100180032B5
:1008910075AC1043AC4043D10275D5A075D4FF436C
:0908A100D10843BA0243AF08225A
:03008B0002001E52
:10001E00C0E0C0D075D000C000E5AC30E01653ACE7
:10002E00FE7451255AF8A6ADE55AC3940750020541
:10003E005A754500E5AC30E10553ACFDC201D00068
:05004E00D0D0D0E0322B
:10081200E4F594F593F592F5917596FFF595F5B299
:10082200F5B1F5B4F5B3F5CAF5C9F5CCF5CBF5E2FA
:03083200F5E122CB
:05000300E580F4FF227E
:030008008FA022A4
:0607C7008B098A0A890B70
:1007CD00E4FFEFC39D50182001FDAB09AA0AA90B48
:0F07DD008F827583001200A7F5ADD2010F80E364
:0107EC0022EA
:1007ED00E545C394025003054522B2C6750C00754C
:1007FD000D00750E51855A0F7B007A00792112027A
:05080D00D4E4F55A22BD
:10087600E544C394025003054422B2C67B007A00C5
:0B0886007949AD5912000EE4F559222B
:0100190022C4
:1006CC00A2B6B3E4335401FFAE09EE54FE4FF50964
:1006DC00A2B7B3E433540125E0FFAE09EE54FD4F4D
:1006EC00F509A2C1B3E433540125E025E0FFAE09BE
:1006FC00EE54FB4FF509A2C2B3E433540133333348
:10070C0054F8FFAE09EE54F74FF509A2C3B3E43326
:10071C005401C454F0FFAE09EE54EF4FF509A2C4D6
:10072C00B3E4335401C43354E0FFAE09EE54DF4F4D
:10073C00F509AF09EF54BFF509AF09EF547FF5097F
:02074C00AF09F3
:01074E002288
:10074F00858308120812120891D2ACD2AF1206CCD0
:10075F008F48AF48EFC4135401F546E548540FF5E1
:10076F0047750CFF750D07750EC77B007A00792151
:10077F001200538546218547221200038F48854872
:10078F0023B2C61207ED7B007A007921120471E5BE
:10079F00416004C2C58002D2C5AF241200081208FE
:1007AF007612001A1200197F647E001208AA055CE7
:0807BF00E55C70C5055B80C11B
:060835008B168A178918DA
:10083B00E4FFFEEEC39D5013AB16AA17A9188E82C8
:0B084B007583001200A72FFF0E80E84D
:01085600227F
:100053008B098A0A890B90001DE4F5F01201C09008
:100063000021E4F5F01201C0AB0CAA0DA90EC003E8
:10007300C002C001AB09AA0AA90B90001812021D05
:01008300225A
:100857008B198A1A891BAB1CAA1DA91EC003C002CB
:0F086700C001AB19AA1AA91B90001812021D227A
:0602D4008B098A0A890B68
:1002DA00AB0CAA0DA90E8B108A118912E50F6404C2
:1002EA006003020470E50F14FD120835AB10AA1161
:1002FA00A9129000031200A76F6003020470AB09F1
:10030A00AA0AA90B12008E7003020394AB10AA1159
:10031A00A91212008E6469705FAB09AA0AA90B9030
:10032A0000041200A7FFAB10AA11A9129000011233
:10033A0000A76F7043AB09AA0AA90B900017041211
:10034A00011990001DE4F5F01201C0AB10AA11A921
:10035A00129000021200A7FFAB09AA0AA90B90008B
:10036A00041200A7FD7C00E92405F9E43AFAE92D14
:10037A00F9EC3AFAEF120107AB09AA0AA90B9000A5
:10038A00061200A7900003020119AB10AA11A912C4
:0A039A0012008E6449600302047033
:1003A400E50B240FF9E4350A850913F5148915AB17
:1003B40009AA0AA90B9000011200A7FFAB10AA1109
:1003C400A9129000011200A76F600302047090004C
:1003D400021200A7AB09AA0AA90B90000312011983
:1003E40090001BE4F5F01201C0AB13AA14A9157414
:1003F40069120107AB09AA0AA90B9000011200A710
:10040400AB13AA14A915900001120119AB09AA0A89
:10041400A90B9000021200A7AB13AA14A91590000F
:1004240002120119AB09E50B240FF9E4350AFA7D30
:1004340003120835AB13AA14A915900003EF120197
:1004440019AB09E50B240FF9E4350AFAC003C0021D
:10045400C001AA0AA90B9000181201ED89828A83AF
:0C046400D001D002D0030D7C0012027AFF
:010470002269
:06058A008B0C8A0D890EA6
:10059000E9240FF9E43A8B0FF5108911A90E9000A8
:1005A000021200A790000B120119AB0FAA10A9119B
:1005B0007449120107AB0CAA0DA90E900004120099
:1005C000A7AB0FAA10A911900001120119AB0CAA38
:1005D0000DA90E9000041200A7FF7E00E9240AF97D
:1005E000E43AFAE92FF9EE3AFA12008EAB0FAA10AC
:1005F000A911900002120119AB0CE50E240FF9E4C9
:10060000350DFA7D03120835AB0FAA10A911900021
:1006100003EF120119AB0CE50E240FF9E4350DFAC6
:10062000C003C002C001AA0DA90E9000181201ED6E
:1006300089828A83D001D002D0030D7C0002027A25
:100471008B098A0A890B12008E70030205359000E0
:100481002112013B540F600302057A9000171200FC
:10049100A7602090001F7401120119900020120022
:1004A100A76044AB09AA0AA90B90002074FF1200AF
:1004B100D48034AB09AA0AA90B90001DE475F001A0
:1004C10012017390001D12013BD3940AE5F09400D0
:1004D1004015AB09AA0AA90B900020741412011946
:1004E10090001FE4120119AB09AA0AA90B9000019F
:1004F1001200A7D39400500302057A9000047401FE
:100501001200D49000011200A7FF9000041200A76E
:10051100D39F400EAB09AA0AA90B900004740112E3
:100521000119AB09AA0AA90B900017E412011912CB
:10053100058A8045AB09AA0AA90B90001BE475F056
:100541000112017390001B12013BD394C8E5F09492
:10055100004010AB09AA0AA90B9000207464120193
:10056100198016AB09AA0AA90B9000201200A760F6
:100571000890002074FF1200D4AB09AA0AA90B90BD
:090581000021E475F00102017390
:09000E008B098A0A890B8D0C2272
:01001A0022C3
:10064C0002074FE493A3F8E493A34003F68001F26E
:10065C0008DFF48029E493A3F85407240CC8C333AF
:10066C00C4540F4420C8834004F456800146F6DF7E
:10067C00E4800B01020408102040809008BDE47E49
:10068C00019360BCA3FF543F30E509541FFEE49373
:10069C00A360010ECF54C025E060A840B8E493A33A
:1006AC00FAE493A3F8E493A3C8C582C8CAC583CA65
:1006BC00F0A3C8C582C8CAC583CADFE9DEE780BE1D
:0108CD00002A
:10008E00BB010689828A83E0225002E722BBFE0270
:09009E00E32289828A83E49322A3
:1000A700BB010CE58229F582E5833AF583E022500E
:1000B70006E92582F8E622BBFE06E92582F8E22258
:0D00C700E58229F582E5833AF583E4932272
:1000D400BB010FF8E58229F582E5833AF583E02830
:1000E400F0225009C58229F8E58226F622BBFE09D2
:1000F400C58229F8E22582F222F8EA2583F583E90C
:030104009328221B
:10010700BB010689828A83F0225002F722BBFE01D7
:02011700F322D1
:10011900F8BB010DE58229F582E5833AF583E8F01C
:10012900225006E92582C8F622BBFE05E92582C8C8
:02013900F222B0
:10013B00BB0110E58229F582E5833AF583E0F5F002
:10014B00A3E0225009E92582F886F008E622BBFEDF
:10015B000AE92582F8E2F5F008E222E5832AF58325
:08016B00E993F5F0A3E99322EA
:10017300BB010DC58229C582C5833AC58302027CB2
:100183005011C58229F808E5F026F618F5F0E58246
:1001930036F622BBFE11C58229F808E225F0F5F0F8
:1001A300F218E23582F222F8E58229F582E5832A04
:0D01B300F58374019325F0F5F0E4933822F4
:1001C000F8BB0111E58229F582E5833AF583E8F071
:1001D000E5F0A3F0225009E92582C8F608A6F0222E
:0D01E000BBFE09E92582C8F2E5F008F22215
:1001ED00BB010DE58229F582E5833AF5830202A470
:1001FD005007E92582F8020292BBFE07E92582F835
:10020D000202B6E58229F582E5833AF5830202C83A
:10021D00BB0120E58229F582E5833AF583D0F0D044
:10022D00E0F8D0E0F9D0E0FAD0E0FBE8C0E0C0F0B3
:10023D000202AD5018E92582F8D083D082D0E0F9C2
:10024D00D0E0FAD0E0FBC082C08302029BBBFE1857
:10025D00E92582F8D083D082D0E0F9D0E0FAD0E061
:09026D00FBC082C0830202BF2223
:060276008A838982E47313
:10027C00C5F0F8A3E028F0C5F0F8E582158270020D
:06028C001583E038F022AA
:09029200E6FB08E6FA08E6F92291
:09029B00EBF608EAF608E9F62288
:0902A400E0FBA3E0FAA3E0F9225B
:0902AD00EBF0A3EAF0A3E9F02252
:0902B600E2FB08E2FA08E2F92279
:0902BF00EBF208EAF208E9F22270
:0C02C800E493FB740193FA740293F92292
:00000001FF
